:0400000000000428D0
:080008008A110A120728853055
:1000100083160313860064205E2002308312860656
:100020006E30FF00003030200C28080083120313CC
:10003000A8007F08A700A90129082707AA00280807
:10004000AB000318AB0A2A0884000008AC000319AF
:100050002F282C08502083120313A90A1C280800FB
:1000600083120313A2007F08A100A3012308210724
:10007000A4002208A5000318A50A422825088A0022
:10008000240882003E2083120313A60026080319C9
:100090004F282608502083120313A30A362808008D
:1000A00083120313A000831203130C1E5328831220
:1000B000031320088312031399000800831203130B
:1000C0008C1E5E281A0808008130831603139900DD
:1000D00024309800903083129800080048346F3420
:1000E0006C346134203463346F346D346F342034B5
:1000F000653473347434613473342E342E342E34B6
:020100000034C9
:02400E00FF3F72
:00000001FF
